:020000020000FC
:0200000005C336
:0200040018954D
:02000800189549
:02000C00189545
:02001000189541
:02001C00189535
:0200240018952D
:0200280089C08D
:02002C00A7C06B
:02003000189521
:02004000189511
:0200440062C098
:02004800189509
:02004C00189505
:02005000189501
:020054001895FD
:020058001895F9
:02005C001895F5
:020060001895F1
:020064001895ED
:020068001895E9
:02006C001FC0B3
:020070001895E1
:020074001895DD
:020078001895D9
:02007C001895D5
:020080001895D1
:020084001895CD
:020088001895C9
:02008C001895C5
:020090001895C1
:020094001895BD
:020098001895B9
:02009C001895B5
:0200A0001895B1
:0200A4001895AD
:0200A8001895A9
:1000AC002FB6DF2DCE2DF49BD6300000F499D7302F
:1000BC0039F418607091C9007F7B7093C9001DC022
:1000CC000E94730E7991FD2EEC2EF09914C0D091F4
:1000DC002F01D03881F00F921F92D79F17FE02C0CC
:1000EC007FEF05C0712D703810F07FEF02C0000C4F
:1000FC00771F1F900F907093CE002FBE18952FB6C0
:10010C000260DD2009F0DA94CA9409F010C07AE09C
:10011C00C72E0460F09B06C000005D9B02C05D987A
:10012C0001C05D9ABA9409F002C0B72E0160E5CF08
:10013C002FB67091E10073FF19C07091E100777ECA
:10014C007093E10077277093E9007091EB00716078
:10015C007093EB0070E07093EC0070E07260709341
:10016C00ED007091F00078607093F0002FBE189540
:10017C002FB68F937091F40070FF07C070E07093EE
:10018C00E9007091E80073FD0DD07091F40072FDE0
:10019C00D6D1F79B04C07091F40073FD13D28F91EC
:1001AC002FBE1895EF93FF937091F100709305019A
:1001BC007091F100709306017091F1007093080139
:1001CC007091F100709309017091F10070930A0124
:1001DC007091F10070930B017091F10070930C0110
:1001EC007091F10070930D017091E800777F70931E
:1001FC00E80070910501F79B06C0713209F47DC0CF
:10020C00713A09F470C0717619F0713009F00BC0B5
:10021C0070910601703041F07530A9F0763039F1EB
:10022C00793009F485C0E0C077277093F1007093A2
:10023C00F1007091E8007E7F7093E8007091E80007
:10024C0072FFFCCFD6C0709108017F777093E300EA
:10025C007091E8007E7F7093E8007091E80070FF69
:10026C00FCCF7091E30070687093E300C2C0709192
:10027C000901713029F0723069F0733021F1B4C08A
:10028C00F79B03C0EEEEFCE102C0ECEBFDE1D49178
:10029C00B3D0AFC0D0910C01D03049F070910D01AA
:1002AC00703029F4F79BD536F799D33420F0F79BAF
:1002BC00D5E6F799D3E4F79B03C0E0E4FDE111C068
:1002CC00EAECFDE10EC070910801772319F4E4E823
:1002DC00FDE106C0713019F4E6E9FDE101C084C00E
:1002EC00D491F6D086C070910601713209F07CC0B1
:1002FC00E2EBFDE1D7E0ECD07CC0709106017032EE
:10030C0051F47091E80072FFFCCF7091E8007B7F94
:10031C007093E80003C0723209F066C07091E80077
:10032C007E7F7093E8007091E80070FFFCCF61C095
:10033C00F79BC2E0F799C3E0C093E9007091EB0022
:10034C007E7F7093EB007091ED007D7F7093ED00DC
:10035C00CA9591F771E07093E9007091EB007160B0
:10036C007093EB0071E87093EC0070E37260709323
:10037C00ED0077277093F00072E07093E9007091B4
:10038C00EB0071607093EB0070E87093EC0070E31D
:10039C0072607093ED007091F00074647093F000D3
:1003AC00F79B14C073E07093E9007091EB007160DF
:1003BC007093EB0071EC7093EC0070E172607093D1
:1003CC00ED007091F00071607093F00077277093DE
:1003DC00E9007091E8007E7F7093E8007091E8006E
:1003EC007170E1F3F69A05C07091EB007062709336
:1003FC00EB00FF91EF91089570910D01772331F48B
:10040C0070910C017D1708F4D72FCC277091E80060
:10041C0072FD94C075917093F100DA95C395C83054
:10042C00A9F77091E8007E7F7093E8007091E80066
:10043C007570E1F37091E80072FD80C0EF93FF934B
:10044C008F939F935F935527F1E0E8E00E943B0B5D
:10045C00802D0E943B0B902D813411F4933211F0BE
:10046C00982B41F481E48093F10083E28093F100B6
:10047C005FEF04C08093F1000092F1000E943B0BEF
:10048C00802D0E943B0B902D863321F4903011F47B
:10049C00552321F40E943B0B002061F486E390E08D
:1004AC00F79B92E80000F79B86E38093F100909312
:1004BC00F10006C0F79B01968093F1009093F10038
:1004CC005F919F918F91FF91EF91CCE0D45014C02C
:1004DC0070910D01772329F470910C017D1708F4AC
:1004EC00D72FCC277091E80072FD28C0A895759184
:1004FC007093F100DA95C39577E07C2349F4709101
:10050C00E8007E7F7093E8007091E8007570E1F36D
:10051C00D03041F77091E800747009F00AC0709106
:10052C00E8007E7F7093E800A8957091E80072FF58
:10053C00FBCF7091E8007B7F7093E80008955F9388
:10054C0072E07093E9007091E80072FF39C070910D
:10055C00E8007B7F7093E80010FD32C07091F200D0
:10056C00772309F1D62DC72D5091F1005993D53031
:10057C0011F4D2E0C0E06D2E7C2E6F93572D662DBA
:10058C00681430F009F005C0791410F049F001C07E
:10059C006D5F59196809623018F05F3B08F0116003
:1005AC006F917A9509F710FD0BC07091E8007B7F75
:1005BC007093E80000007091E8007F777093E8007A
:1005CC005F9108955F9373E07093E9007091E80078
:1005DC0070FF14C0707A7093E80011FF09C0C0EC72
:1005EC00D1E070910F0159915093F1007A95D9F7A0
:1005FC001D7F7091E8007F777093E8005F910895FC
:10060C00F89491E09EBF9CEF9DBF88279FEF84B923
:10061C0095B987B998B98AB99BB98DB99EB980BB80
:10062C0091BB002711272227CC24C394BC2CF1E0CA
:10063C00E0E099279193F130E8F3539A5B9A37995C
:10064C0007C0F1E0E8E055270E94460BED30D9F7E2
:10065C00519A59980E94C00C9927909380009CE065
:10066C009093810092E081E79093890080938800B9
:10067C0092E090936F0090B7906890BF8EE19EE0EF
:10068C00809360009093600099279EBB0E942F0B73
:10069C0090931B010E94720B0E94550BA895F69B20
:1006AC00FDCF0E945D0B0E942F0B90931B01559A5E
:1006BC00209A28985D98F1E0E4E00E943B0B0092B0
:1006CC002301A895A8954427332718600E94C00CD5
:1006DC000E94140C0E943B0A0E94350EF49B07C02A
:1006EC000FD7F6F79A35E1F7DBD11F78F9CF08D79A
:1006FC00F6F7F3D0FCCF6F938F939F93982F609165
:10070C00110163956093110197FF50C0903F29F43C
:10071C002160217F90931201DCC0973F19F5613065
:10072C00A9F1623081F097E0909310019091130140
:10073C0090931201909114019093130197EF909361
:10074C001401207F95C096E09093100190911301B5
:10075C009093120197EF90931301992790931401A2
:10076C00207F86C090931201943FE8F0983F89F067
:10077C009E3F79F09A3F69F09B3F59F09C3F49F0BE
:10078C009F3F39F0963F29F0247F9FC097EF9093BD
:10079C0012019927909313019093140195E0909373
:1007AC001001207F65C02160217F93C020FD0CC00B
:1007BC00207F909312019FE09093100199279093C2
:1007CC0013019093140154C021FD1EC0909313018A
:1007DC0099279093140190911201913F79F0933FD6
:1007EC0069F0907F903C21F0903D11F0226071C037
:1007FC009295909310012160217F3AC092E09093E2
:10080C0010012160217F34C020FF5FC022FD18C081
:10081C009093140123FF02C024605BC090911201DD
:10082C00923F49F0903FF9F092959F709093100190
:10083C002160217F1DC093E090931001207F18C090
:10084C0020FF43C022FF41C080911301809312010D
:10085C0080911401809313019093140194E0909370
:10086C001001297F05C094E090931001297F286026
:10087C00F894000091E09093E900A8959091E8001D
:10088C0090FFFBCF9E7B9093E8009091100190938A
:10089C00F100909112019093F100909113019093BB
:1008AC00F100909114019093F1009091E8009E7FDB
:1008BC009093E80000009091E8009F779093E800F7
:1008CC00789499279093110104C099279093110162
:1008DC00207F9F918F916F910895F09B05C0A895F3
:1008EC009A3509F0089584C09A3519F4D9D01F7837
:1008FC009EC0F0999CC0963511F4F8D198C09335F0
:10090C0011F4DED194C0943508F064C0903408F032
:10091C0026C0933219F40E946D0689C0943219F4E2
:10092C000E944A3F84C0963219F40E94483F7FC00F
:10093C009B3219F40E94B20B7AC09C3211F4D0D1C4
:10094C0076C09D3219F40E94C70B71C09D3311F40F
:10095C00D5D16DC09F3319F40E94AD0868C0903496
:10096C0019F40E94100C63C0913411F458D25FC07A
:10097C00923411F40DD25BC0933419F40E94FB0530
:10098C0056C0943419F40E948C0C51C0973419F44D
:10099C000E9408074CC0983419F40E94BA0647C04C
:1009AC009D3411F4FED143C09E3439F490913B0137
:1009BC00923010F00E9435073AC0903511F445D2B0
:1009CC0036C0913519F40E94820731C0923511F46A
:1009DC0069D22DC0943511F46BD329C0973519F415
:1009EC000E94C30624C0983519F40E946C3F1FC0A6
:1009FC00953511F4B8D01BC09E3519F40E944C3FAC
:100A0C0016C09F3519F40E945F3F11C09C3719F432
:100A1C000E94AB0C0CC09E3719F40E94D30B07C07C
:100A2C009D3009F435C09A3011F0903209F40895D4
:100A3C00F79909C080912301806C0E9481038FE398
:100A4C000E94810305C08FE30E94E20A0E94E10A22
:100A5C0026D692E0692E892E90E0792E992EF89464
:100A6C000000E2E0E093E900E091E800EB7FE09326
:100A7C00E8000000E091E800EF77E093E8001E78D2
:100A8C00F098077E91E09EBF9CEF9DBF789426CE98
:100A9C00F49908950000F79B08950E94E10A0895C7
:100AAC009AE0D92EA8952CD5DD2019F4F09BC0CF57
:100ABC000895CEF79A35A1F31F79913A81F010641D
:100ACC00923A69F09AE0D92EA895DD2039F018D524
:100ADC00E6F79A3529F3953A09F0F7CF27C0086065
:100AEC001061F09AAA27A0933B01A0933C01A0931C
:100AFC003E01BB27F7E0E0E096E0D92EDD20B1F017
:100B0C00FFD4E6F7F93008F491931196BB23A1F3C7
:100B1C00B23011F015FDF0CFA13071F716FF04C003
:100B2C0015FD02C01062E8CF953A41F08AE544D534
:100B3C0081EC42D585EA40D5077F0895F7E0E0E0E7
:100B4C00B5E0A0E091919D93F49903C0B630D1F734
:100B5C0002C0B730B9F78AE52FD581EC2DD585EADF
:100B6C002BD5077F08953F925F936F930F9300628D
:100B7C00F198F2989FE786EE0E94240B98D066F4C9
:100B8C00332E832FF19A38D5F19891D02EF4832FF0
:100B9C00F19A32D5F19801C026C0532F9FE78CEE05
:100BAC000E94240B84D06EF4832FF19A0E94020BC6
:100BBC00F198432E7CD02EF4832FF19A1DD5F19809
:100BCC0001C011C0F1E0E8E05BD5532D59D5532F8E
:100BDC0057D5542D55D55AE553D5B9D20F916F91A0
:100BEC005F913F9008950C941E059FE78EEC26D5DF
:100BFC008AE3E2D482E004D30EF03BC00F7E3A309D
:100C0C0010F4832F04C081E3D7D4832F8A50805DE6
:100C1C000E94E20A532F552361F1513150F55F9335
:100C2C009FE78CED0BD59FE78EEC08D58AE3C4D4F7
:100C3C0082E0E6D25F910EF01CC00F7E3A3010F4C9
:100C4C00832F04C081E3B8D4832F8A50805D0E9427
:100C5C00E20A0F7E351769F480E2AED48FE6ACD48D
:100C6C008BE6AAD48DE0A8D4F1E0E4E05A9508D53F
:100C7C0008950C941E0508609170F92F0E94860A45
:100C8C00EEF7E92F9F2B09F4F2E00E949B0B0E94D8
:100C9C00860AEEF7077F092E309127014091280133
:100CAC000E94B90D3093270140932801089582E0EA
:100CBC00E0D226F4442311F468940895E89408953E
:100CCC0083E00E94060916F40E949C0D089583E0AF
:100CDC000E94060926F40E949C0D0E94B30D0895F3
:100CEC000E94F70856F40E949E0B03C00E94F7085E
:100CFC0026F430932A010E94B30D089583E00E94DC
:100D0C0006090EF00895442371F580912701909106
:100D1C0028018F3F08F027C08F939F93E82FF92F5E
:100D2C00FE5F008000922A01019680932701909328
:100D3C002801332389F03F938F939F930E94B30D27
:100D4C009F918F913F910196803031F080932701D4
:100D5C00909328013A9569F79F91909328019F9160
:100D6C0090932701089564CE0E94F7080EF0089521
:100D7C00309331010E94F60C08950E94F7080EF092
:100D8C00089530953695309333010E94F60C0895F2
:100D9C000E94F7080EF00895309332010E94F60C71
:100DAC00089583E00E9406090EF00895393C08F07E
:100DBC003FCE30933001343611F430E820C0393B4B
:100DCC0010F096E015C0363910F095E011C03837A8
:100DDC0010F094E00DC0353510F093E009C03233BB
:100DEC0010F092E005C03F3010F091E001C099275F
:100DFC00532F56955695350F390F08F43FEF309316
:100E0C002F01089583E00E9406090EF008954423F3
:100E1C0029F43A3518F430933A0110C009CE83E026
:100E2C000E9406090EF008954423C1F73A35B0F735
:100E3C003130A1F330933B01332309F031E030938F
:100E4C003E01332730933C01089583E00E9406094C
:100E5C000EF0089530933D0130933E0108953F9379
:100E6C004F93EF93FF9380913D0180933E018091CE
:100E7C003C019927442730913A01380F3A3508F054
:100E8C0033270E945C0CFF91EF914F913F91809121
:100E9C003C01839590913B01891709F48827809335
:100EAC003C01089583E00E9406090EF00895442346
:100EBC0009F021C0313808F030E883E70E94E20ADB
:100ECC0090912601809125010E948E0986E70E944F
:100EDC00E20AF5E0E0912501EA9581910E947D09F5
:100EEC00E03031F03A9521F08CE20E94E20AF5CF25
:100EFC000E94E10A08959CCD0F921F9283E40E94F8
:100F0C00E20A88E40E94E20A8DE30E94E20A8091E0
:100F1C002501682F909126010E948E0980E20E9483
:100F2C00E20AF0912801E0912701FE5F508186E4EE
:100F3C000E94E20A89E60E94E20A8EE60E94E20A18
:100F4C008DE30E94E20A852F0E947D0980E20E94B7
:100F5C00E20AF0912801E09127016E2F51915F93E5
:100F6C0084E50E94E20A88E50E94E20A8DE30E9471
:100F7C00E20A852F0E947D0980E20E94E20A82E546
:100F8C000E94E20A8DE30E94E20A5F91852F909104
:100F9C002F01903841F0899F812D803810F08FEF10
:100FAC0002C0000C881F0E947D0980E20E94E20AA8
:100FBC006F3F91F187E40E94E20A8DE30E94E20AFE
:100FCC00819190912F01903841F0899F812D80382B
:100FDC0010F08FEF02C0000C881F0E947D0980E288
:100FEC000E94E20A6E3FC1F082E40E94E20A8DE3A5
:100FFC000E94E20A808190912F01903841F0899FE4
:10100C00812D803810F08FEF02C0000C881F0E94D9
:10101C007D0980E20E94E20A0F938DE40E94E20AAD
:10102C0086E40E94E20A8DE30E94E20A0F7B809123
:10103C0030010E94F00985E20E94E20A80E20E94DF
:10104C00E20A83E40E94E20A83E50E94E20A8DE34D
:10105C000E94E20A80913A010E94F0098FE20E94FC
:10106C00E20A80913B010E94F0098FE20E94E20AA1
:10107C0080913D018F770E94F00980E20E94E20A84
:10108C0084E50E94E20A8DE30E94E20A80912B0122
:10109C000E94F0098EE20E94E20A80912C010E94CB
:1010AC00F0090F918DE00E94E20A1F900F900895B5
:1010BC00992790932B0190932C0183E0A1D00EF0F3
:1010CC00B7CC423008F0B4CC5F9355279927442312
:1010DC0011F099E156E0332361F03A3018F03A50B0
:1010EC009395FBCF350F3A3010F03A5093955F91B2
:1010FC0002C0352F5F91903210F09FE139E0909350
:10110C002B013A3008F039E030932C0100244427AD
:10111C00990F892F990F990F890F041E890F041E9F
:10112C00890F041E890F041E890F041E890F041ECB
:10113C00880F001C330F432F330F330F340F44270A
:10114C00830F041E00922D0180932E0108959EE7BB
:10115C008CEE0E94240B9FE784E20E94240B9FE7F5
:10116C0086EE0E94240BF1E0E8E00E943B0B902DF0
:10117C000E943B0B802D892B11F0802D02C091E435
:10118C0083E20F930062F19A37D2F198892F34D20F
:10119C009FE78CEE0E94240BF1E0EAE00E943B0BEF
:1011AC00802D0E943B0B502D0E943B0B002011F018
:1011BC00952F02C086E390E0F79902C092E886E38F
:1011CC00582F892FF19A18D2F198852F15D28DE0CE
:1011DC00F3D19FE784E80E94240B0F9108950C949F
:1011EC001E0506FF04C082E044D03EF403C083E039
:1011FC0007D01EF4442311F4689408950C941E0532
:10120C007FD1F6F7332744278F9302C079D1F6F7B5
:10121C009D3039F19A3029F1903278F0B9F39C3243
:10122C00A9F39E3299F39033E0F09734D0F49134D3
:10123C0020F49A33B0F452D016F00C941E05330FF0
:10124C00441F532F642F330F441F330F441F350F8C
:10125C00461F6627390F461F8A95C1F668948F91F1
:10126C00089500619F91891711F4E894089568948A
:10127C0008958F933327442743D1F6F79D3089F394
:10128C00973F11F49DE0EDCF9032E8F0A9F3903345
:10129C0040F3973430F7913410F49A3310F718D098
:1012AC0016F00C941E05330F441F330F441F330FDD
:1012BC00441F330F441F6627390F461F8A95E1F6EA
:1012CC0068948F9108950C941E05913470F002C0AF
:1012DC00913420F0973448F4975305C0903328F09C
:1012EC0090539A3010F468940895E89408959F935D
:1012FC00992706FF0AC08F9384E2F7995DD100000D
:10130C00F79BF9D98F9166D001C064D09F91089555
:10131C000F930F7D5F936F933F92582F992369F131
:10132C009732B0F011F4503198F087E2382E60E12A
:10133C008827931540F011F4561728F08395006216
:10134C00561B9309F6CF8063F79936D1F79BD3D907
:10135C0083E0382E68EE8827931540F011F4561769
:10136C0028F083950062561B9309F6CF806305FF26
:10137C0004C0F79921D1F79BBED98827332464E6A2
:10138C00992311F4561728F083950062561B930984
:10139C00F7CF806305FF04C0F7990ED1F79BABD94B
:1013AC0088276AE0561720F083950062561BFACF07
:1013BC00806305FF04C0F799FFD0F79B9CD9852F5C
:1013CC008063F799F9D0F79B96D93F906F915F9115
:1013DC000F9108950F9306FF1BC09F93982F829532
:1013EC008F7005FD41F0805D8A3308F0895FF799B5
:1013FC00E3D0F79B80D9892F8F70805D8A3308F0FA
:10140C00895FF799D9D0F79B76D99F910F91089561
:10141C009F935F93982F8827943660F054E680E36F
:10142C008395951B9436E0F79F93F799C5D0F79B5E
:10143C0062D99F91882311F49A3068F05AE080E3C6
:10144C009A3018F08395951BFBCF9F93F799B4D0E6
:10145C00F79B51D99F91892F805DF799ADD0F79B60
:10146C004AD95F919F910F910895A89501FF44C0AF
:10147C000D7F992790933701F09918C012FD0E94A7
:10148C00030E02FF13C00B7F90913B01992371F067
:10149C0080913D01882351F080913E01882331F0E9
:1014AC008A9580933E0111F40E94350700FF1BC002
:1014BC000E7F14FD05C00000F09B02C0F0985D98F3
:1014CC00C8D080911B01891771F05D9AF8940E9425
:1014DC00550B81E08EBF8CEF8DBF7894A8950E9440
:1014EC005D0B0C94590380911501882329F08A9582
:1014FC008093150109F45D9813FD0E94440E089524
:10150C008F93EF93FF93B1DF04FF04C090913801E8
:10151C000F7E3CC0E894F82DE92D972D9E1721F4F1
:10152C00962D9F1709F443C09191F53011F4F2E018
:10153C00E0E08F2E9E2E5F936F93572D662D6814CF
:10154C0030F009F005C0791410F0E1F001C06D5FC6
:10155C0059196809623010F0503BA0F410FF12C00A
:10156C001E7FF8940000F2E0F093E900F091E8009F
:10157C00FB7FF093E8000000F091E800FF77F09318
:10158C00E80078946F915F9190933801F79B07C0B6
:10159C0003FD05C09B3718F4913608F090520F7E6E
:1015AC006894F09904C0E9E1E09315015D9AFF910C
:1015BC00EF918F9108958DE08F93F894000081E066
:1015CC008093E900A8958091E80080FFFBCF8E7B8B
:1015DC008093E8008F918F938093F1008091E800C5
:1015EC008E7F8093E80000008091E8008F778093D5
:1015FC00E80078948F9108958F9305FD02C080E2E6
:10160C00DBDF8F918F9382958F70805D8A3308F02A
:10161C00895FF19908C0F29B02C0803329F08033B6
:10162C0011F4F19B80E2C8DF8F918F938F70805DF6
:10163C008A3308F0895FC0DF8F910895FF93EF9391
:10164C00FC018591882311F0B7DFFBCFEF91FF915F
:10165C0008951D9B05C09927F79AF498F39804C038
:10166C009FEFF79AF49AF39A089503D00094319669
:10167C000895F2BDE1BD002403940FBA00B408959F
:10168C00509502D031960895A895F894F2BDE1BD1D
:10169C0050BDFA9AF99AF999FECF789408959F93D0
:1016AC009AEFA8950AD09A95E1F79F910895F7DFE4
:1016BC00F6DFF5DFF4DFF3DF08959F9398EC9923C1
:1016CC0049F09F939F919F939F9100000000000011
:1016DC009A95F5CF9F910895002491E09093D700AF
:1016EC0090EB9093D80000009F7D9093D800000061
:1016FC0090629093D80090E199BD926099BD99B594
:10170C0090FFFDCF9091D8009F7D9093D8009927A2
:10171C009093E00098E09093E20092E0692E892E7D
:10172C0090E0792E992E78940895FB5F3197089567
:10173C00E0912501F0912601FF2361F43196E093AD
:10174C002501F09326010E949B0BF0932801E09356
:10175C00270108950C941E05F0912801E0912701B2
:10176C005081FE5F0080902D9F3F49F003940082D2
:10177C0000922A01F250951719F4008201C0F25020
:10178C000895F0912801E09127015081FE5F0080BF
:10179C00902D9923A1F30A94EACF82E00E940609C6
:1017AC00C6F53A3510F00C941E0513FFFECFAF931F
:1017BC00BF93EF93FF933F93F4E2F30FEE27A0E078
:1017CC00B7E09BE5909337010E94023FE0E89BE570
:1017DC00909337010E94023F9927909337013F91D4
:1017EC00332399F4F1E0E0E050912D010E94460B77
:1017FC0050912E010E94460B5FEF06FD55270E946B
:10180C004A0B3196522F0E94460BFF91EF91BF91DC
:10181C00AF91089582E00E940609DEF73A3510F088
:10182C000C941E053323B1F4F1E0E0E00E943B0B75
:10183C0000922E010E943B0B00922D010E943F0B47
:10184C000F7B01FE006431960E943B0B902D907F24
:10185C002F70292BAF93BF93EF93FF93F4E2F30F09
:10186C00EE27A0E0B7E0A895059000940D92A0306B
:10187C00D9F7F5E0E0E0B7E0A0E0A8950C90508136
:10188C00501559F080912E0190912D01992321F43E
:10189C00882311F4008201C080D131961196F63064
:1018AC0061F7FF91EF91BF91AF9108953A3510F028
:1018BC000C941E05AF93BF93EF93FF93F4E2F30FD9
:1018CC00EE27A0E0B7E0A895059000940D92A13802
:1018DC00D9F7F5E0E0E0B7E0A0E0A8950C905081D6
:1018EC00501559F080912E0190912D01992321F4DE
:1018FC00882311F4008201C050D131961196E13841
:10190C0061F7FF91EF91BF91AF9108959FE78CED37
:10191C0095DE0E94860AEEF79F7D943411F00C94AC
:10192C001E058DE049DEF894F5E0E0E0B7E0A0E0BC
:10193C0099279193F49905C09D93F630D1F778943B
:10194C000895F730B1F7789408959FE78CED76DE23
:10195C000E94860AEEF79C3711F00C941E05F89441
:10196C00F1E0E4E055278CDEA2DEA1DEA0DE8DE006
:10197C000E94E20AF894F5E0E0E099279193FB309D
:10198C00E9F70F7B1F7B992790932A0190932B01EA
:10199C0090932C0190932D0190932E0190932601FE
:1019AC0082E380933A0190933B019093390184E157
:1019BC0080933D01939590932501909333019FEF74
:1019CC009093320190E890932F0194E6909330011C
:1019DC0095E09093280190E09093270178940895D6
:1019EC00309131013B3238F4330F5FEF531B330F1F
:1019FC00632F882742C0353580F43B52432F4695E0
:101A0C00469546956BEA330F630F330F3395339539
:101A1C005CEA531B541B882730C0303840F43555D2
:101A2C00330F6FEF631B330F832F552726C03A3AC2
:101A3C0080F43058432F4695469546958BEA330FE4
:101A4C00830F330F339533956CEA631B641B552757
:101A5C0014C0353D40F43A5A330F8FEF831B330FCC
:101A6C00532F66270AC0355D5BEA330F530F330FD4
:101A7C00339533958AEA831B66271F929091330125
:101A8C009F779923C1F09F3709F490E84FEF451BDE
:101A9C00499F412D000C441F540F4FEF461B499F8B
:101AAC00412D000C441F640F4FEF481B499F412DE3
:101ABC00000C441F840F909132019F3F69F0969562
:101ACC00599F512D000C551F699F612D000C661FED
:101ADC00899F812D000C881F1F9060933501809386
:101AEC003601309125014091260150932A010E9424
:101AFC00B30D0090350100922A010E949E0B0E94AA
:101B0C00B30D0090360100922A010E949E0B0E9498
:101B1C00B30D3093250140932601E32FF42F0E943F
:101B2C009B0BF0932801E09327010895442329F09F
:101B3C00423088F4332379F402C0332361F03093BC
:101B4C00250140932601E32FF42FEFDDF0932801BC
:101B5C00E093270108950C941E05F0912801E09163
:101B6C00270100902A0100922A01F0932801E093AA
:101B7C0027015081501509F40EC0FE5F0082F2500F
:101B8C0080912E0190912D01992321F4882311F439
:101B9C00008201C002D078940895501908F4519530
:101BAC00002480912E0190912D010AD0FD5F90832D
:101BBC00F39580838827F3958083F55014600895FE
:101BCC004F923324441861E1001C551F6A9551F45F
:101BDC009695879583199409802D952F08F4019675
:101BEC004F900895331C441C381A490A20F4380EBF
:101BFC00491E8894E9CF0894E7CF5F936F933F9287
:101C0C00F5E0E0E01B7F8081FE5F9081891711F485
:101C1C00F2501DC0F3955081F3956081F39530809F
:101C2C00360E08F453953082891740F4850F20F056
:101C3C00981710F0146009C0892F07C0851B20F07D
:101C4C00891710F0146001C0892FF55080833196EC
:101C5C00E03009F0D8CF3F906F915F910895599A79
:101C6C0093E09093CC009091C8009D7F9093C80016
:101C7C0099279093C9009EE09093CA000E94630B31
:101C8C00F8949091C900977B9093C9005B98539AF4
:101C9C0078940E94630B5B9A14D01FD0F89495E053
:101CAC00F92EEE249091C90098649093C90099275D
:101CBC009093CE00177F789408959F9392E00C94A4
:101CCC00650B9F9390E10C94650B9F9390EB0C9498
:101CDC00650B9F9390E00C94650B9F9394E00C9490
:101CEC00650B12011001020000080E01000000013A
:101CFC0009024300020100803109040000010202C4
:101D0C00000005240010010524010300042402072F
:101D1C000524060001070583031000400904010097
:101D2C00020A0000000705810240000107050202BB
:101D3C004000010009024300020100803109040047
:101D4C00000102020000052400100105240103001B
:101D5C000424020705240600010705830310004034
:101D6C0009040100020A000000070581024000403E
:101D7C00070502024000000A120355006E00200005
:101D8C004B006E006F0077006E001C035500530073
:101D9C0042002D00530069006D0070006C0065005E
:101DAC0044006D00780000C2010000000800000033
:101DBC0012010002010000080E01000100010902DD
:101DCC0065000201008031090400000001010000DF
:101DDC0009240100010900010109040100020103A9
:101DEC000000072401000141000624020101000645
:101DFC002402020200092403010301020100092448
:101E0C0003020401010100090581024000000000E9
:101E1C00052501010309050202400000000005250B
:041E2C0001010100AF
:0223FE000000DD
:10780000FFFFFF00FFFFFFFFFFFFFFFFFFFFFFFF87
:06781000FFFFFF5060FFC6
:10790000FFFFFF4040FFFFFFFFFFFFFFFFFFFFFF05
:06791000FFFFFF00FFFF76
:107A0000FFFFFFFF00FFFFFFFFFFFFFFFFFFFFFF85
:067A1000FFFF4040FFFFF4
:107B0000FFFFFFFF5060FFFFFFFFFFFFFFFFFFFFD3
:067B1000FFFF00FFFFFF74
:107C0000FFFFFFFFFF00FFFFFFFFFFFFFFFFFFFF83
:067C1000FFFF60FF60FFB2
:107D0000FFFFFF60FF60FFFFFFFFFFFFFFFFFFFFC1
:067D1000FFFFFFFF00FF72
:107E00000C9406035F938F939F93EF93FF93F43249
:107E100020F4FE3710F00C941E05F999FECF9091D6
:107E200037019B3511F00C941E059927909337016B
:107E3000F89493E00E94423F91E10E94423F80E427
:107E40000D901D900094109491E00E94423F329654
:107E50008A95B1F7FF91EF91EF93FF9395E00E9420
:107E6000423F91E10E94423F87B786FF04C091E103
:107E70000E94423FF9CF7894FF91EF919F918F91AB
:107E80005F91089557B750FDFDCF97BFE8950895CE
:107E90000F7B0895006408950E94F7087EF4F09126
:107EA0002801E0912701FE5F9081930F08F49FEF76
:107EB000092E90932A01F2500E94B90D08950E9454
:107EC000F708E6F7F0912801E0912701FE5F908125
:107ED000931B70F79927ECCFE0E0F5E0A0E0B7E066
:107EE00091919D93F630E1F71B7F08950D73696DB5
:107EF000706C65205553422F444D5820496E74656F
:107F0000726661636520666F722041726475696E86
:107F10006F204C656F6E6172646F202876312E3150
:107F20003429000020286329323031352D323120A8
:107F3000572E536368656D6D6572740D00004A7548
:107F40006D706572204F46463A41534349495F631D
:107F50006D64536574202B204D696E69444D582C17
:107F600032353663680D4A756D706572204F4E3A32
:107F70004D4944495F636D645365742C32353663F3
:107F8000680D00004A756D706572204F46463A4193
:107F9000534349495F636D64536574202B204D69D9
:107FA0006E69444D582C32353663680D4A756D70D4
:107FB0006572204F4E3A6F6E6C79204D696E694440
:107FC0004D58206275742035313263680D004D497B
:107FD000444920636828312D3136290020526570CC
:107FE0006561742000005649443D0000205049441A
:027FF0003D0052
:00000001FF
